:020000040000FA
:06000000A2EF1EF0120049
:0600080004EF08F01200F5
:060018000CEF08F01200DD
:06100000A2EF1EF0120039
:021006001200D6
:0610080022EF08F01200C7
:01100E0000E1
:0610180098EF08F0120041
:02101E000300CD
:101020009C3D000060000000380000008A3D000088
:10103000E4000000120000000E1000004C0100004F
:0410400001000000AB
:0C104400DACFE4FFE2CFDAFFE9CFE4FFEF
:10105000EACFE4FFF6CFE4FFF7CFE4FFF5CFE4FFFC
:10106000F3CFE4FFF4CFE4FFFACFE4FF00EE00F0AB
:10107000140EE80403E3EECFE4FFFBD700EE14F018
:10108000080EE80403E3EECFE4FFFBD7E6529EA48C
:1010900002D09E948B8A9EA00AD09E908BC01CF09A
:1010A0001D6A1C50CF6E00018A51CE6E8B9A9EA293
:1010B00011D09E920001862B000E8723FE0ED88051
:1010C0008855FF0E895503E2886B896B03D0882B06
:1010D000000E8923F2B4F294A1A406D0A1943CECB2
:1010E00011F00001010E856FE55200EE1BF0080EB5
:1010F000E80403E3E5CFEDFFFBD700EE13F0140E99
:10110000E80403E3E5CFEDFFFBD7E5CFFAFFE5CF3A
:10111000F4FFE5CFF3FFE5CFF5FFE5CFF7FFE5CF30
:10112000F6FFE5CFEAFFE5CFE9FFE5CFDAFF1100F3
:10113000D8CFE4FFE0CFE4FFE46EDACFE4FFE2CF04
:10114000DAFFE652E552E5CFDAFFE550E5CFE0FF02
:10115000E5CFD8FF1000D9CFE6FFE1CFD9FF040ECD
:10116000E126A0949B8CDCEC0DF08B880001866B53
:10117000876BE2EC10F027EC19F00001A76BBADAEC
:1011800079DBD0B2FFD7C7DA00019E6B9F6BA16BF2
:10119000A06B9A6B020EDB6A030EDB6ADE6ADD6A05
:1011A000DECF14F0DDCF15F0D890155004E6030E15
:1011B000145C000E155815E2DFCFE6FF78EC0DF059
:1011C000E552146E156AD950020FE96EDACFEAFFC4
:1011D0001450EE261550ED22DF2A010E01E3DB2A22
:1011E000DFD7020EDBCF08F0030EDBCF09F0020ED3
:1011F00008C0DBFF030E09C0DBFFDE6ADD6ADECF5D
:1012000014F0DDCF15F0020EDBCF16F0030EDBCFAE
:1012100017F015501718E8AE02D0173404D0165046
:10122000145C1750155807E236EC19F0DF2A010E4E
:1012300001E3DB2AE4D700019969800EE66ECF0E48
:10124000E66E4F0EE66E5DD8E552E552E5520001BE
:10125000A8B9938EA8BB938AA8BD7F86D08E3B0E7B
:10126000606EA284A084F28E0001020E865D000EE4
:10127000875901E2F9D7866B876BC7D851EC0EF01E
:1012800039DAF2D7040EE15C02E2E16AE552E16E7E
:10129000E552E7CFD9FF1200CD901200CD801200A9
:1012A000CD50010B00D01200D9CFE6FFE1CFD9FF1E
:1012B000FE0EDB50EA6A980FE96E000EEA22FC0E81
:1012C000DBCFEEFFFD0EDBCFEDFFE552E7CFD9FF21
:1012D0001200D9CFE6FFE1CFD9FFFE0EDB50EA6A5C
:1012E000980FE96E000EEA22EECF14F0EFCF15F062
:1012F00014C0F3FF15C0F4FF00D0E552E7CFD9FFCB
:101300001200D9CFE6FFE1CFD9FFC6DFFD0EDBCF5C
:101310008AF0FE0EDBCF8BF00001FF0ED8808A57DB
:101320008B57FD0EDBCF14F0FE0EDBCF15F0010E58
:101330000F0B05E0D89015321432E806FBE114508B
:1013400000018A258C6F15508B218D6F8BC014F096
:10135000156A1450CF6E8A51CE6E8DC014F0156A86
:101360001450BF6E8C51BE6EE552E7CFD9FF12000C
:101370000001912B910506E10001010EA76F000EFF
:1013800043D040D00A0E915D19E10001030EA76F12
:101390008E0EE66E540EE66E060EE66E85DFE552A4
:1013A000E552E5520A0EE66EE66A080EE66E7CDF4E
:1013B000E552E552E552000E27D024D0140E915D7F
:1013C00019E10001070EA76F1A0EE66E470EE66ED2
:1013D000060EE66E69DFE552E552E5520A0EE66E4C
:1013E000E66A080EE66E60DFE552E552E552000E51
:1013F0000BD008D01E0E915D05E10001070EA76F0E
:10140000010E02D0000E00D01200D9CFE6FFE1CFCE
:10141000D9FF020EE1267FD900019551070A01E1AB
:10142000B0D0010A01E1A8D0020A01E19DD0070A6B
:1014300001E18BD0020A46E0040A35E00C0A29E0FB
:10144000010A1DE0080A01E0A3D000019969B85122
:10145000146E156A153404E21450C808000E1554B1
:1014600007E28B880001030E956F0001A76B06D081
:10147000A25104E18B880001080E956F89D078DFB6
:10148000000906E00001010E956F936B0001996B56
:101490007FD06EDF000906E00001050E956F936BAB
:1014A0000001996B75D00001B851146E156A15349E
:1014B00004E21450C808000E155404E30001060E9F
:1014C000956F66D08B880001B851146E156A15347B
:1014D00004E21450C808000E155403E20001050E82
:1014E000956F0001A251000824E200019351146E8F
:1014F000156A153404E21450C808000E155416E29B
:10150000070E956FC9DEE90EE66E5E0EE66E060EFC
:10151000E66ECADEE552E552E5521E0EE66EE66A5A
:10152000080EE66EC1DEE552E552E5520001932B4E
:101530000BD0995107E100019351000803E200012B
:10154000010E996F0001936B23D00001A251000896
:1015500008E20001932B9351050802E2040E956FF7
:1015600002D00001936B14D00001A25104E10001EC
:10157000090E956F936B0CD00001070EA76F8B9827
:1015800007D00001070EA76FA25101E18B9800D090
:101590000001A551320803E2010EA26F01D0A26B37
:1015A000D9EC19F0080EE66E94DEE552F3CF14F094
:1015B000F4CF15F0000ED8801454000E15543DE2FF
:1015C000060EE66E86DEE552F3CF14F0F4CF15F08A
:1015D00000019651141802E19751151803E160DEDD
:1015E000000815E359DE060EE66E73DEE552F3CF12
:1015F00096F0F4CF97F0800EE66E96C0E6FF97C0A7
:10160000E6FF7FDEE552E552E55248DE15D0080ED2
:10161000E66E5FDEE552F3CF14F0F4CF15F014065A
:10162000000E155A14C0E6FF15C0E6FF080EE66E60
:101630003BDEE552E552E5520CD0080EE66E49DE7F
:10164000E552F3CF14F0F4CF15F01450151001E16A
:1016500023DE000E0001E76E9919E8AE02D099353D
:1016600003D0E750D880995537E29B5100081EE21D
:101670000001942B0A0E945D18E3040EE66E29DE39
:10168000E552F3CF14F0F4CF15F0010E1426000E3E
:10169000152214C0E6FF15C0E6FF040EE66E04DE58
:1016A000E552E552E5520001946B02D00001946BC3
:1016B0000001A8B907D0010EA815000802E28A8E21
:1016C00001D08A9EA8BB07D0020EA815000802E22E
:1016D0008A8A01D08A9A04D0A8A98A9EA8AB8A9A3D
:1016E000020EE15C02E2E16AE552E16EE552E7CF0B
:1016F000D9FF12000001A7A102D08B9C01D08B8CD6
:10170000A7A302D08B9E01D08B8EA7A502D08A9C66
:1017100001D08A8C1200E66AEBD9E5520001A36F72
:10172000020EE66EE5D9E5520001A56F030EE66EE6
:10173000DFD9E5520001B86F12DAF3CFB9F0F4CF78
:10174000BAF00001BB6BBC6BA951E824146E156A9A
:10175000E80E1426030E1522166A176A15AE02D07B
:1017600016681768B90EE96E000EEA6E14C00BF029
:1017700015C00CF016C00DF017C00EF0EECF06F03D
:10178000EECF07F0EECF08F0EFCF09F0DBEC1DF065
:1017900005C0EDFF04C0EDFF03C0EDFF02C0EFFF89
:1017A000E80E0B6E030E0C6E0D6A0E6AB9C006F0E1
:1017B000BAC007F0BBC008F0BCC009F064EC1EF072
:1017C00006C0B9F007C0BAF008C0BBF009C0BCF051
:1017D000200E0B6E500E0C6E0D6A0E6AB9C006F02C
:1017E000BAC007F0BBC008F0BCC009F0DBEC1DF0CC
:1017F00002C0B9F003C0BAF004C0BBF005C0BCF031
:10180000A00E0B6E860E0C6E010E0D6E0E6AB9C028
:1018100006F0BAC007F0BBC008F0BCC009F064EC29
:101820001EF006C0B9F007C0BAF008C0BBF009C08E
:10183000BCF0B9C0A4F00001A8A905D081AE02D0C7
:10184000A88101D0A891A8AB14D0A8AD0DD0040EEA
:10185000E66E4ED9E5520001A66FA6517F0802E25E
:10186000A88301D0A89305D081AA02D0A88301D073
:10187000A8931200D9CFE6FFE1CFD9FF020EE126EF
:10188000DE6ADD6ADECF14F0DDCF15F0D89015509A
:1018900004E6200E145C000E155815E2DFCFE6FFBB
:1018A0008CD8E552E66EDECFE9FFDDCFEAFF980E79
:1018B000E926000EEA22E552E750EF6EDF2A010E1C
:1018C00001E3DB2ADFD7FF0E0001985D01E10AD8B2
:1018D000020EE15C02E2E16AE552E16EE552E7CF19
:1018E000D9FF1200D9CFE6FFE1CFD9FF020EE126E2
:1018F000DE6ADD6ADECF14F0DDCF15F0D89015502A
:1019000004E6200E145C000E15581AE2DECFE9FF43
:10191000DDCFEAFF600EE926000EEA22EF50E66E08
:10192000DECFE9FFDDCFEAFF980EE926000EEA22BE
:10193000E552E750EF6EDF2A010E01E3DB2ADAD72A
:101940000AD8020EE15C02E2E16AE552E16EE5527C
:10195000E7CFD9FF1200D9CFE6FFE1CFD9FF020EC2
:10196000E126DE6ADD6ADECF14F0DDCF15F0D89017
:10197000155004E6200E145C000E155814E2DECF5C
:10198000E9FFDDCFEAFF980EE926000EEA22EF50CC
:10199000E66EDFCFE6FF24D8E552E552DF2A010EDE
:1019A00001E3DB2AE0D7020EE15C02E2E16AE552E4
:1019B000E16EE552E7CFD9FF1200D9CFE6FFE1CFC4
:1019C000D9FFFE0EDB50A96EAA6AA69EA69CA68031
:1019D000A6B0FED7A85000D0E552E7CFD9FF12003D
:1019E000D9CFE6FFE1CFD9FFFE0EDB50A96EAA6A80
:1019F000FD0EDB50A86EA69EA69CA684F29EF28CDD
:101A0000550EA76EAA0EA76EA682A6B2FED7F28EBC
:101A1000F28CA694E552E7CFD9FF1200F29E550E44
:101A2000A76EAA0EA76EA682A6B2FED7A694120033
:101A3000D9CFE6FFE1CFD9FF020EE126FD0EDBCFC5
:101A400014F0FE0EDBCF15F0000E14263E0E15220C
:101A500014C0DEFF15C0DDFFF86ADECF14F0DDCF65
:101A600015F015C014F0156A1450F76EDECF14F09F
:101A7000DDCF15F01450F66E0900F55000D0146E4D
:101A8000020EE15C02E2E16AE552E16E1450E552B9
:101A9000E7CFD9FF1200D9CFE6FFE1CFD9FF020E81
:101AA000E1266492646ADE6ADD6ADECF14F0DDCF7F
:101AB00015F0D890155004E6FF0E145C000E155872
:101AC0000CE2E868E85004E0E80600D000D0FAD75D
:101AD000DF2A010E01E3DB2AE8D7FF00020EE15CFA
:101AE00002E2E16AE552E16EE552E7CFD9FF12006A
:101AF000D9CFE6FFE1CFD9FFE652FE0EDB50040A54
:101B000015E0070A10E0010A0BE0030A06E0010AEB
:101B100001E00FD0040EDF6E0DD0050EDF6E0AD08F
:101B2000060EDF6E07D0070EDF6E04D00B0EDF6EE1
:101B300001D0DF6ADF5000080BE2C16ADF50040DFC
:101B4000F3500109C26EC282C2B2FED7C45002D0A5
:101B5000000E00D0E552E552E7CFD9FF1200080E83
:101B6000C16E150EC26EC282C2B2FED7C450166ECE
:101B7000176AD89016361736D89016361736FC0ED8
:101B80001616030E1716C350186E196A060ED89053
:101B900019321832E804FBE1030E1816000E19166C
:101BA00016501824146E17501920156E14C0F3FF28
:101BB00015C0F4FF00D0120002D8E2EF10F00001CF
:101BC000010E846F200EE66EE66AE66A980EE66EF7
:101BD000000EE66E88EC1EF0146E050EE15E1450E9
:101BE0000F0E946EFB0E826EDB0E8B6E100E936EDC
:101BF000B00E816E400E8A6EF00E7E6E7F6AC16AF4
:101C00003E0EC06E8B880001806B816B826B836B94
:101C1000010E846FD66AD76AB192B196B19AB19823
:101C2000B19EB184CD9CCD92CD8ECD9ACD88CD96EE
:101C3000CD84CD908A6B800E8B6F8BC014F0156AAB
:101C40001450CF6E8A51CE6EBD86BD94BD82BD90BC
:101C5000C00EBF6EBE6ACA8CCA8ACA88CA96CA80BB
:101C6000CA82FA0ECB6EB990B992B994B996B98876
:101C7000D58CD59AD598D584D592D590D5969D807A
:101C80009D829D84F28AD08EF1849F809F829F8462
:101C9000A282F28EF28CD59ECA84E00EBA6E40EF1C
:101CA0001EF0D9CFE6FFE1CFD9FF080EE1260001F3
:101CB000845100E0200E0001BF5D03E36450020B7D
:101CC00001E0FAD100018051811102E1000E08D03B
:101CD00080C0E9FF81C0EAFFEF50800B01E0010EF8
:101CE000000901E0E9D102013651AA0A01E1ABD1B4
:101CF000C80A01E1A1D1320A01E103D1200A01E1C0
:101D000000D11D0A30E0200A2EE0CC0A06E0010ACC
:101D100001E0BFD10001846BBCD1810E766F000160
:101D20008251831102E1000E08D082C0E9FF83C016
:101D3000EAFFEF50800B01E0010E000913E1400EB5
:101D4000E66E760EE66E020EE66E010EE66EE66E4C
:101D50008BEC18F0146E050EE15E1450F3CF82F098
:101D6000F4CF83F096D16D0E766F720E375D4CE135
:101D7000720E776F38C278F239C279F2DE6ADD6AA4
:101D8000DECF14F0DDCF15F03951000115AE02D0D1
:101D9000D89003D0145C000E155835E2020138517A
:101DA000186E196ADE501824166EDD501920176E51
:101DB000D890175004E6200E165C000E175823E248
:101DC0003851146E156ADE501424E96EDD5015206A
:101DD000EA6E980EE926000EEA22EF50E66EDECF9C
:101DE000E9FFDDCFEAFF040EE926000EEA22760EB7
:101DF000E926020EEA22E552E750EF6EDF2A010ED5
:101E000001E3DB2ABDD759D0770E375D56E1720E5C
:101E1000776F38C278F239C279F2020EDB6A030EAC
:101E2000DB6A020EDBCF14F0030EDBCF15F0395165
:101E3000000115AE02D0D89003D0145C000E1558E6
:101E40003CE202013851186E196A020EDB50182468
:101E5000166E030EDB501920176ED890175004E64B
:101E6000200E165C000E175828E2020EDBCFE9FFA9
:101E7000030EDBCFEAFF040EE926000EEA22360E3F
:101E8000E926020EEA22EF50E66E3851146E156A0A
:101E9000020EDB501424E96E030EDB501520EA6EAF
:101EA000980EE926000EEA22E552E750EF6E020E88
:101EB000DB2A030E01E3DB2AB4D700018251831130
:101EC00002E1000E08D082C0E9FF83C0EAFFEF50B4
:101ED000800B01E0010E000913E1400EE66E760E64
:101EE000E66E020EE66E010EE66EE66E8BEC18F004
:101EF000146E050EE15E1450F3CF82F0F4CF83F040
:101F0000C8D0700E766F720E375D72E1720E776F09
:101F100038C278F239C279F23AC27AF238C216F08F
:101F200016C017F0166A3951196A000F186EFF0EA5
:101F3000192216501814146E17501914156EFF0E2E
:101F40001416000E1516060E14C0DBFF070E15C082
:101F5000DBFF040EDB6A050EDB6A040EDBCF14F038
:101F6000050EDBCF15F002013A51000115AE02D08B
:101F7000D89003D0145C000E15583AE2040EDBCF63
:101F800016F0050EDBCF17F0D890175004E6400E80
:101F9000165C000E17582CE2040EDBCF16F0050E6F
:101FA000DBCF17F0060EDB501624146E070EDB5045
:101FB0001720156E14C0E6FF15C0E6FF39DDE552A7
:101FC000E552E66E040EDBCFE9FF050EDBCFEAFF3C
:101FD000E926000EEA22760EE926020EEA22E552F2
:101FE000E750EF6E040EDB2A050E01E3DB2AB5D7BE
:101FF00000018251831102E1000E08D082C0E9FF86
:1020000083C0EAFFEF50800B01E0010E000913E1ED
:10201000400EE66E760EE66E020EE66E010EE66E7F
:10202000E66E8BEC18F0146E050EE15E1450F3CFE3
:1020300082F0F4CF83F02DD0E668E668D1DCE5527B
:10204000E55229DD26D0550E766F000182518311AD
:1020500002E1000E08D082C0E9FF83C0EAFFEF5022
:10206000800B01E0010E000913E1400EE66E760ED2
:10207000E66E020EE66E010EE66EE66E8BEC18F072
:10208000146E050EE15E1450F3CF82F0F4CF83F0AE
:1020900000D0400EE66E360EE66E020EE66EE66A82
:1020A000010EE66E8BEC18F0146E050EE15E145016
:1020B000F3CF80F0F4CF81F0080EE15C02E2E16A38
:1020C000E552E16EE552E7CFD9FF1200120012008F
:1020D00012001200B3EF1CF012001E0EE66E010E8D
:1020E000E66EE5EC17F0E552E552400EE66E360E70
:1020F000E66E020EE66EE66A010EE66E8BEC18F0F6
:10210000146E050EE15E1450F3CF80F0F4CF81F031
:10211000120064840001080EBD6F070EBE6FBD077C
:10212000000EBE5BBD51BE11FAE164941200D9CF1E
:10213000E6FFE1CFD9FFFD0EDBCF08F0FE0EDBCFCF
:1021400009F0010E081801E1095033E0E8680818A9
:1021500002E1E86809182BE0030E081801E10950B4
:1021600024E0040E081801E109501DE0020E0818D1
:1021700001E1095016E0170E081801E109500FE0BF
:10218000160E081801E1095008E0150E081801E1C3
:10219000095001E010D0A1DF0FD09EDF0DD09ADFF3
:1021A0000BD096DF09D092DF07D091DF05D091DF09
:1021B00003D0000001D000D0010E00D0E552E7CFDF
:0421C000D9FF120031
:0C21C400D9CFE6FFE1CFD9FFE652020EB2
:1021D00001014C5D02E24C2B00D00F015F6B626A83
:1021E000648C649C5C6B000EE66EE66AE66A540ED4
:1021F000E66E0F0EE66E88EC1EF0146E050EE15EC4
:102200001450DF6ADF50146E156A080E145C000E5D
:10221000155810E2DF50040DF3CFE9FFF4CFEAFFC9
:10222000000EE926020EEA22EE6AEE6AEE6AEE6A15
:10223000DF2AE8D70F01160E536F62A60CD0030EEB
:10224000E66E620EE66E0F0EE66E04EC19F0E552D5
:10225000E552E552F2D70001D26BD76BD86BD96B40
:102260006498080ECA6F020ECB6FC06BBF6BE5524D
:10227000E552E7CFD9FF1200D9CFE6FFE1CFD9FF72
:10228000E652A1940001BF0507E164BA05D0626A75
:1022900060806088020EBF6F6250040B0FE06050D8
:1022A000040B0CE0020EE66E620EE66E0F0EE66E9A
:1022B00004EC19F0E552E552E552E7D864B2A0D03B
:1022C0006250010B1BE06050010B18E07BDF000146
:1022D000040EBF6F0201200E026F020E036F080E84
:1022E000016F006B8C0E0013E66A620EE66E0F0E35
:1022F000E66E04EC19F0E552E552E5526250100B1F
:102300000FE06050100B0CE0A4D8040EE66E620ED5
:10231000E66E0F0EE66E04EC19F0E552E552E5525A
:102320006250400B1DE06050400B1AE0010EE66E5B
:10233000E66A000EE66EE66A020EE66EE66A97EC64
:1023400010F0146E060EE15E1450060EE66E620E7C
:10235000E66E0F0EE66E04EC19F0E552E552E5521A
:102360006250200B04E06050200B01E04ED8625018
:10237000020B13E06050020B10E0010EE66EE66AFD
:10238000000EE66EE66AE668E66897EC10F0146EFA
:10239000060EE15E14500F015F6B040E0001BF5D7D
:1023A00001E22ED060A62CD0DF6A040EDF5C28E2AA
:1023B00062A625D063CFDFF0030EE66E620EE66EF6
:1023C0000F0EE66E04EC19F0E552E552E552780E78
:1023D0000001DF1502E178D810D0000EE66EE66A43
:1023E000DF0EE66E000EE66E010EE66EE66A97EC14
:1023F00010F0146E060EE15E1450DF2AD6D700D01E
:10240000E552E552E7CFD9FF12000F0153A115D0D5
:10241000C2C0E9FFC3C0EAFFEF5080080DE1CAC0A7
:10242000E9FFCBC0EAFFEF50840806E1C2C0E9FF34
:10243000C3C0EAFF8C0EEF6E5391050EE66E620E7E
:10244000E66E0F0EE66E04EC19F0E552E552E55229
:1024500012006084040EE66E620EE66E0F0EE66EEB
:1024600004EC19F0E552E552E5526482000EE66E86
:10247000E66AE66EE66A040EE66EE66A97EC10F02F
:10248000146E060EE15E145012006492000EE66EA9
:10249000E66AE66EE66A030EE66EE66A97EC10F010
:1024A000146E060EE15E1450609462A40CD0020E0D
:1024B000E66E620EE66E0F0EE66E04EC19F0E55263
:1024C000E552E552F2D71200FD0E0001DF1520E1C2
:1024D0007E0EDF15E8407F0B040DF3CFC2F0F4CF82
:1024E000C3F0000EC227020EC323C2C0C4F0C3C093
:1024F000C5F0C475C2C0E9FFC3C0EAFFEF503C0B92
:10250000E842E8420D0802E109D801D02AD805D0F6
:10251000FD0EDF15040801E12DD81200CAC0E9FF45
:10252000CBC0EAFFEF50800B05E0CAC0E9FFCBC08B
:10253000EAFFEF6A0001CE6BCF6BD36BD46BD26B2B
:1025400007D9000EE66EE66AE66EE66A170EE66EDC
:10255000E66A97EC10F0146E060EE15E145054EF2C
:1025600015F0020E0001CF5D03E1B1EC16F001D0D1
:1025700051D81200D9CFE6FFE1CFD9FFE652CAC049
:10258000E9FFCBC0EAFFEF50400B01E0010EDF6E28
:102590000001CA75080EBF5D0DE122C25CFF0F018C
:1025A0005C51000804E20001100EBF6F03D000016F
:1025B000040EBF6FCF0528E1CAC0E9FFCBC0EAFF18
:1025C000020EE926000EEA22280EEE6E020EED6ED5
:1025D0003DDB020E0001CE5D07E1CAC0E9FFCBC0C2
:1025E000EAFF840EEF6E0FD0DF5007E1CAC0E9FFAB
:1025F000CBC0EAFFC80EEF6E06D0CAC0E9FFCBC061
:10260000EAFF880EEF6E01D005D8E552E552E7CF1C
:10261000D9FF1200D9CFE6FFE1CFD9FF030EE126A3
:10262000020E0001CF5D4AE16450100B47E0C2C0CA
:10263000E9FFC3C0EAFFEE52EF50146E156A080EB0
:10264000141801E115503AE1C2C0E9FFC3C0EAFF26
:10265000EF503C0BE842E8420D0830E1C4C0E9FF0E
:10266000C5C0EAFFEF50800B29E1C4C0E9FFC5C037
:10267000EAFF020EE926000EEA22200EEE6E020E9E
:10268000ED6EDF6ADF50146E156A080E145C000EE2
:10269000155813E2DF50EA6A280FE96E020EEA22AB
:1026A000EF50E66EDF50EA6A200FE96E020EEA2272
:1026B000E552E750EF6EDF2AE5D731D0CF6BC4C0CB
:1026C000E9FFC5C0EAFFEE52080EEF6EC4C0E9FF95
:1026D000C5C0EAFF020EE926000EEA22200EEE6EC9
:1026E000020EED6EC4C0E9FFC5C0EAFF8C0EEF6EAE
:1026F000CAC0E9FFCBC0EAFFEF6A040ECA19146E24
:10270000CBC015F0010E14C0DBFF020E15C0DBFFBD
:10271000010EDBCFE9FF020EDBCFEAFFEF6A00011B
:10272000D7AF0CD0DA51DB1107E005D0DBC0FAFFE0
:102730000001DA51F96EFADF0001D79F030EE15C68
:1027400002E2E16AE552E16EE552E7CFD9FF1200FD
:1027500002012051600BE842E842E842E842E842C8
:10276000000901E058D021510C0A54E00B0A43E063
:102770000C0A35E0010A26E00B0A22E0020A20E0FA
:10278000030A1CE0080A10E0010A0CE00F0A08E046
:10279000030A01E03FD00001D28F080EBF6F3BD08B
:1027A000C8D839D06FDB37D00001C00ED06F000E13
:1027B000D16FD281010ED36FD28F2DD014D92BD0EF
:1027C0002BD829D024510001D06FD16BC10ED02756
:1027D000000ED123D281010ED36FD28F1CD0000105
:1027E000D28F02012451EA6AC10FE96E000EEA227B
:1027F00022C2EFFF10D0000EE66EE66AE66EE66AD1
:10280000160EE66EE66A97EC10F0146E060EE15EA8
:10281000145001D000D01200D9CFE6FFE1CFD9FF8C
:10282000040EE1260201220510E120511F0B0009D0
:102830000CE10001D28F030E0201215D04E10001D1
:10284000010EDE6F02D00001DE6B0201225167E152
:1028500020511F0B020863E124510F0B00095FE0B8
:102860000001D28F020124BF10D024510F0BE96E5A
:10287000EA6AD890E936EA36C60EE926000EEA2260
:10288000EECFDEFFEDCFDDFF0FD024510F0BE96E51
:10289000EA6AD890E936EA36CA0EE926000EEA223C
:1028A000EECFDEFFEDCFDDFF030E215D07E1DECFD2
:1028B000E9FFDDCFEAFF840EEF6E31D024510F0B1C
:1028C000156A530F146E0F0E1522020E14C0DBFF93
:1028D000030E15C0DBFF020EDBCFE9FF030EDBCFDB
:1028E000EAFFEE90ED5224AF0DD0DECFE9FFDDCF51
:1028F000EAFFEF6ADF74DECFE9FFDDCFEAFF400ECB
:10290000EF6E0DD0DECFE9FFDDCFEAFF880EEF6E70
:10291000DF74DECFE9FFDDCFEAFFC80EEF6E040EF5
:10292000E15C02E2E16AE552E16EE552E7CFD9FFF0
:102930001200800E0201205D55E10001C00ED26F31
:1029400002012351030A2EE0010A0EE0030A03E00C
:102950000001D26B47D00001520ED06F3A0ED16FFA
:10296000120ED36FD46B3ED02251F66EF76AD89018
:10297000F636F736100EF6263B0EF7220900F5CF95
:10298000D0F00A00F5CFD1F0020E0001F76AD02591
:10299000F66ED151F7220900F5CFD3F00A00F5CF3A
:1029A000D4F020D0030E225D1AE22251F66EF76AAF
:1029B000D890F636F736120EF6263B0EF7220900AF
:1029C000F5CFD0F00A00F5CFD1F0D0C0F6FFD1C0DE
:1029D000F7FF0800F5500001D36FD46B02D000015F
:1029E000D26B00D01200D9CFE6FFE1CFD9FF020EA3
:1029F000E1260201286B296B20511F0B020A12E00D
:102A0000030A0DE0010A01E03BD00001D28F020170
:102A100028810001DE0502E10201288331D0000196
:102A2000D28F2ED00001D28F020124BF10D02451AA
:102A30000F0BE96EEA6AD890E936EA36C60EE92647
:102A4000000EEA22EECFDEFFEDCFDDFF0FD02451E6
:102A50000F0BE96EEA6AD890E936EA36CA0EE92623
:102A6000000EEA22EECFDEFFEDCFDDFFDECFE9FF85
:102A7000DDCFEAFFEF50040B02E0010E286F00D01B
:102A80000001D2AF07D0280ED06F020ED16FD281D5
:102A9000020ED36F020EE15C02E2E16AE552E16EE2
:102AA000E552E7CFD9FF120064980001D2BF4AD0A7
:102AB000D7AF28D0020ECF6FCAC0E9FFCBC0EAFF64
:102AC000EE52EF6ACAC0E9FFCBC0EAFFC80EEF6E54
:102AD000C4C0E9FFC5C0EAFFEE52080EEF6EC4C0E5
:102AE000E9FFC5C0EAFF020EE926000EEA22280E21
:102AF000EE6E020EED6EC4C0E9FFC5C0EAFFC80E5F
:102B0000EF6E1FD0C4C0E9FFC5C0EAFFEE52080E49
:102B1000EF6EC4C0E9FFC5C0EAFF020EE926000E51
:102B2000EA22200EEE6E020EED6EC4C0E9FFC5C0B3
:102B3000EAFF8C0EEF6ECAC0E9FFCBC0EAFF840E3D
:102B4000EF6E83D0D7BF81D0020120AF56D00001F5
:102B5000D3510201265D0001D4510201275904E23C
:102B600026C2D3F027C2D4F071D80001010ECF6F76
:102B7000C4C0E9FFC5C0EAFFEE52080EEF6EC4C044
:102B8000E9FFC5C0EAFF020EE926000EEA22200E88
:102B9000EE6E020EED6EC4C0E9FFC5C0EAFF800E06
:102BA000EF6EC2C0E9FFC3C0EAFFEE52080EEF6E3F
:102BB000C2C0E9FFC3C0EAFF020EE926000EEA2206
:102BC000200EEE6E020EED6EC2C0E9FFC3C0EAFF3A
:102BD000800EEF6ECAC0E9FFCBC0EAFF020EE92605
:102BE000000EEA22280EEE6E020EED6ECAC0E9FF5C
:102BF000CBC0EAFFC80EEF6E28D00001020ECF6FE7
:102C0000CAC0E9FFCBC0EAFFEE52EF6ACAC0E9FFD3
:102C1000CBC0EAFFC80EEF6EC4C0E9FFC5C0EAFF33
:102C2000EE52080EEF6EC4C0E9FFC5C0EAFF020E07
:102C3000E926000EEA22280EEE6E020EED6EC4C0EA
:102C4000E9FFC5C0EAFFC80EEF6E1200D9CFE6FF5C
:102C5000E1CFD9FF020EE1260001080ED35D000E80
:102C6000D4590EE2D3C0DEFFD4C0DDFFCE5103E164
:102C7000010ECE6F04D0CE0502E1020ECE6F03D05E
:102C8000080EDE6EDD6ACAC0E9FFCBC0EAFFEF9234
:102C9000CAC0E9FFCBC0EAFFEF90CAC0E9FFCBC0D2
:102CA000EAFF010EDB50EF12CAC0E9FFCBC0EAFF1A
:102CB000EE52DFCFEFFF000EDB50D35F010EDB5093
:102CC000D45B280EDC6F020EDD6FD2B121D0D9CFDC
:102CD000E9FFDACFEAFFEE50ED1019E0D0C0F6FFC1
:102CE000D1C0F7FFD02B000ED1230800F550E66EBF
:102CF000DCC0E9FFDDC0EAFFDC2B000EDD23E5527E
:102D0000E750EF6EDF06010E01E2DB06E0D71FD0D1
:102D1000D9CFE9FFDACFEAFFEE50ED1018E0D0C0CE
:102D2000E9FFD1C0EAFFD02B000ED123EF50E66EB1
:102D3000DCC0E9FFDDC0EAFFDC2B000EDD23E5523D
:102D4000E750EF6EDF06010E01E2DB06E1D7020E6F
:102D5000E15C02E2E16AE552E16EE552E7CFD9FFBC
:102D60001200D9CFE6FFE1CFD9FF020EE126C2C0A3
:102D7000E9FFC3C0EAFFEE52EFCFDFFFDFCF14F071
:102D800014500001D85D000ED95903E2D8C0DFFF0E
:102D900009D0DF50146E156A1450D85DD86F1550E5
:102DA000D959D96F010EDB6ADF50F36E010EDBCF0C
:102DB000F4FFF350F45C16E2010EDB50EA6A280FD0
:102DC000E96E020EEA22EF50E66ED5C0E9FFD6C0EA
:102DD000EAFFD52B000ED623E552E750EF6E010E29
:102DE000DB2AE2D7000ED880D855000ED95528E24C
:102DF000C4C0E9FFC5C0EAFFEE52080EEF6EC4C0C2
:102E0000E9FFC5C0EAFF020EE926000EEA22280EFD
:102E1000EE6E020EED6EC2C0E9FFC3C0EAFFEF50D6
:102E2000400B07E1C4C0E9FFC5C0EAFFC80EEF6E62
:102E300006D0C4C0E9FFC5C0EAFF880EEF6E18D007
:102E4000C4C0E9FFC5C0EAFF020EE926000EEA226F
:102E5000200EEE6E020EED6EDA51DB1107E005D0AA
:102E6000DBC0FAFF0001DA51F96EFADF0001D79FEB
:102E7000020EE15C02E2E16AE552E16EE552E7CF63
:102E8000D9FF12000001D28F000EE66EE66AE66AF4
:102E9000540EE66E0F0EE66E88EC1EF0146E050EF4
:102EA000E15E1450010EE66EE66AE66AC10EE66E59
:102EB000000EE66E88EC1EF0146E050EE15E1450F6
:102EC00022C2C0F00201225104E10001100EBF6FC6
:102ED00011D00001200EBF6F000EE66EE66AE66EAE
:102EE000E66A150EE66EE66A97EC10F0146E060EB2
:102EF000E15E14501200D9CFE6FFE1CFD9FF020EF8
:102F0000E126000EDE6E020EDD6EFD0EDB50E824C3
:102F1000166EFE0EDB50040DF3501624040DF35014
:102F2000146E156A020E0F0B05E0D890153214329C
:102F3000E806FBE1D89014361536D89014361536CD
:102F4000D9CFE9FFDACFEAFF1450EE261550ED2273
:102F5000DECFE9FFDDCFEAFFEF9EFD0EDB500FE194
:102F6000FE0EEA6ADB34FE0BEA36E96EC60EE9268F
:102F7000000EEA22DECFEEFFDDCFEDFF0ED0FE0E1B
:102F8000EA6ADB34FE0BEA36E96ECA0EE926000E69
:102F9000EA22DECFEEFFDDCFEDFFDECFE9FFDDCFB2
:102FA000EAFFEF9CDECFE9FFDDCFEAFF040EE92662
:102FB000000EEA22EF8C020EE15C02E2E16AE552C9
:102FC000E16EE552E7CFD9FF1200D9CFE6FFE1CF9E
:102FD000D9FF020EE126FE0EDB50156A530F146E68
:102FE0000F0E152214C0DEFF15C0DDFFDECFE9FF96
:102FF000DDCFEAFFFD0EDBCFEFFFDBA407D0E66AF3
:10300000FE0EDBCFE6FF77DFE552E552FD0EDBA2D9
:1030100008D0010EE66EFE0EDBCFE6FF6CDFE55258
:10302000E552020EE15C02E2E16AE552E16EE55230
:10303000E7CFD9FF1200D9CFE6FFE1CFD9FF020ECB
:10304000E126FE0EDB5020E1C4C0E9FFC5C0EAFF67
:10305000EE52080EEF6EC4C0E9FFC5C0EAFF020ED3
:10306000E926000EEA22200EEE6E020EED6EC4C0BE
:10307000E9FFC5C0EAFF8C0EEF6ECAC0E9FFCBC006
:10308000EAFF840EEF6E3DD0FD0EDB50E824166E95
:10309000FE0EDB50040DF3501624040DF3CF14F094
:1030A000F4CF15F0000E1426020E152214C0DEFF18
:1030B00015C0DDFF840E146EDECFE9FFDDCFEAFF21
:1030C0001450EF12FD0EDB50E824166EFE0EDB509E
:1030D000040DF3501624010F040DF3CF14F0F4CFB8
:1030E00015F0000E1426020E152214C0DEFF15C0C6
:1030F000DDFF840E146EDECFE9FFDDCFEAFF145052
:10310000EF12020EE15C02E2E16AE552E16EE55285
:10311000E7CFD9FF1200D9CFE6FFE1CFD9FF020EEA
:10312000E126FD0EDB500FE0FE0EEA6ADB34FE0BFB
:10313000EA36E96ECA0EE926000EEA22EECFDEFF7D
:10314000EDCFDDFF0ED0FE0EEA6ADB34FE0BEA3671
:10315000E96EC60EE926000EEA22EECFDEFFEDCFC5
:10316000DDFFDECFE9FFDDCFEAFF020EE926000E2C
:10317000EA22FB0EDBCFEEFFFC0EDBCFEDFFDECF56
:10318000E9FFDDCFEAFFEE52FA0EDBCFEFFF400E94
:10319000146EDECFE9FFDDCFEAFF1450EF16880E84
:1031A000146EDECFE9FFDDCFEAFF1450EF12FD0E03
:1031B000DB500CE0FE0EEA6ADB34FE0BEA36E96E09
:1031C000CA0EE926000EEA22EF740BD0FE0EEA6A60
:1031D000DB34FE0BEA36E96EC60EE926000EEA2263
:1031E000EF74DECF14F0DDCF15F014C0F3FF15C07F
:1031F000F4FF020EE15C03E200D0E16AE552E16E09
:10320000E552E7CFD9FF1200D9CFE6FFE1CFD9FFD2
:10321000010EF36EFC0EDB5004E0D890F336E806A6
:10322000FCE1F350E81C146EFD0EDBCFE9FFFE0E4F
:10323000DBCFEAFF1450EF16E552E7CFD9FF1200BB
:1032400005D0646A606A0001BF6B00D01200000103
:10325000BF510BE1646A606A64B602D06486FCD731
:0C3260000001010EBF6F160E616E12001F
:04326C00D9CFE6FFD1
:10327000E1CFD9FF040EE1260B0E1F0BE4C014F0C2
:10328000E5C015F0E6C016F0E7C017F007E0D890EB
:103290001436153616361736E806F9E1E40EE96EEF
:1032A000000EEA6EEE50141AEE50151AEE50161A71
:1032B000EE50171A14C0DFFF010E15C0DBFF020E1F
:1032C00016C0DBFF030E17C0DBFFE8C0E4F0E9C067
:1032D000E5F0EAC0E6F0EBC0E7F0ECC0E8F0EDC0E6
:1032E000E9F0EEC0EAF0EFC0EBF0F0C0ECF0F1C0B6
:1032F000EDF0F2C0EEF0F3C0EFF0F0C014F0F1C06A
:1033000015F0F2C016F0F3C017F0130ED890173274
:10331000163215321432E806F9E1F00EE96E000EAD
:10332000EA6EEE50141AEE50151AEE50161AEE50C0
:10333000171AD9CFE9FFDACFEAFFEECF18F0EECFB8
:1033400019F0EECF1AF0EFCF1BF0080ED8901B3219
:103350001A3219321832E806F9E1D9CFE9FFDACF8B
:10336000EAFFEE50181AEE50191AEE501A1AEE50E3
:103370001B1A145018180001F06F15501918F16F2E
:1033800016501A18F26F17501B18F36FF0C006F0A2
:10339000F1C007F0F2C008F0F3C009F0040EE15CE0
:1033A00003E200D0E16AE552E16EE552E7CFD9FFD2
:1033B0001200D9CFE6FFE1CFD9FF050EE1261E0EA0
:1033C000DF6E000E0001E76E9919E8AE02D0993564
:1033D00003D0E750D880995501E3C1D0FF0E995D25
:1033E00001E1BDD099510001F45D03E00001A76B3C
:1033F0009A6B00019A51040DF3CF14F0F4CF15F03D
:1034000014C0E6FF15C0E6FF18EC0DF0E552E552DA
:103410000101416F040EDB6A030EF36E040EDBCF75
:10342000F4FFF350F45C27E2040EDB50166E176ACB
:1034300000019A51040DF3501624146EF450172015
:10344000156E010E1426000E152214C0E6FF15C0DD
:10345000E6FF18EC0DF0E552E552E66E040EDB5087
:10346000EA6A420FE96E010EEA22E552E750EF6E7A
:10347000040EDB2AD1D701014151FE0A5EE0CE0ADB
:1034800059E0010A57E0030A55E0010A53E0070A30
:1034900051E0010A4FE0030A4DE0010A4BE00F0A38
:1034A00049E0780A47E0010A45E0030A43E0010ADF
:1034B00041E0070A3FE0010A3DE0030A3BE0010A60
:1034C00039E00F0A37E04E0A32E0160A2DE0010A11
:1034D0002BE0030A29E0010A27E0330A25E0010A6C
:1034E00023E0030A21E0010A1FE0260A1AE0010A8C
:1034F00015E0070A10E00A0A0BE0080A07E0010AD3
:1035000001E023D042C19AF0DF061FD0DF6A1DD050
:1035100040D8DF061AD0D8D8DF6A17D02CD8DF06FB
:1035200014D030D8DF6A11D04BD8DF060ED0C9D8FE
:10353000DF060BD0F4D8DF0608D00001996BA16B31
:10354000A06BDF6A070EA76F00D0DF50000807E20C
:103550000001040E865D000E875901E24AD799C02A
:10356000F4F0050EE15C02E2E16AE552E16EE5523B
:10357000E7CFD9FF120043C19FF042C19EF0000186
:103580009A2B120043C1A1F042C1A0F000019A2B76
:1035900012006CDE020E0B6E0C6A0D6A0E6A64EC91
:1035A0001EF0010E021805E1035003E1045001E191
:1035B000055003E142C19AF002D043C19AF01200D3
:1035C000D9CFE6FFE1CFD9FF030EE126010141513A
:1035D000F00BE83AE76E010EE7CFDBFF41510F0B2E
:1035E000E76E020EE7CFDBFF010EDB50020A06E0BA
:1035F000030A01E00CD043C1DFFF09D04351EA6A5E
:10360000980FE96E000EEA22EFCFDFFF00D0020E26
:10361000DB50030A3BE0010A27E0030A14E0010A39
:1036200001E045D04251EA6A980FE96E000EEA22A5
:10363000EFCF14F0DF50145C03E144C19AF002D0E4
:1036400000019A2B34D04251EA6A980FE96E000EBD
:10365000EA22EFCF14F0DF50145C03E044C19AF08B
:1036600002D000019A2B23D04251EA6A980FE96EEA
:10367000000EEA22EFCF14F0DF50D880145403E29A
:1036800044C19AF002D000019A2B11D04251EA6A4B
:10369000980FE96E000EEA22EFCF14F0DF50145CB1
:1036A00003E244C19AF002D000019A2B00D0030E2D
:1036B000E15C02E2E16AE552E16EE552E7CFD9FF53
:1036C000120042C19AF012000001F55116E143C107
:1036D00014F014C015F0146A000E1416FF0E15161F
:1036E000010142511424456F000E1520466F476BAF
:1036F000486B0001010EF56F11D0F5050FE10101D6
:103700004507000E465B475B485B45514611471134
:10371000481104E144C19AF00001F56B1200D9CFC1
:10372000E6FFE1CFD9FF090EE12601014151F00B7F
:10373000E83AE76E010EE7CFDBFF41510F0BE76E72
:10374000020EE7CFDBFF010EDB50040A06E0070A9A
:1037500001E00CD043C1DFFF09D04351EA6A980F62
:10376000E96E000EEA22EFCFDFFF00D0020EDB5041
:10377000080A01E1E3D00F0A01E1D7D0010A01E113
:10378000CBD0030A01E1BCD0010A01E1AAD0070AAB
:1037900070E0010A3DE0030A0CE0010A01E0D7D025
:1037A0004251EA6A980FE96E000EEA22DFCFEFFF7E
:1037B000CED0DFCF16F04251EA6A980FE96E000EC4
:1037C000EA22EF501624146E156A000E1522030E1D
:1037D00014C0DBFF040E15C0DBFF030EDBCF14F0BB
:1037E000040EDBCF15F0153404E21450FF08000E70
:1037F000155404E2030EDB68040EDB6A4251EA6AE8
:10380000980FE96E000EEA22030EDBCFEFFF9FD088
:103810004251EA6A980FE96E000EEA22EF50166EE6
:10382000176ADF50186E196A1850165C146E19501A
:103830001758156E050E14C0DBFF060E15C0DBFF12
:10384000050EDBCF14F0060EDBCF15F00001800E65
:10385000151404E0050EDB6A060EDB6A0101425115
:10386000EA6A980FE96E000EEA22050EDBCFEFFF41
:103870006ED04251EA6A980FE96E000EEA22EF50CC
:10388000166E176ADF50146E156A14C008F015C062
:1038900009F016C00DF017C00EF013EC1EF0070E65
:1038A00006C0DBFF080E07C0DBFF070EDBCF14F0FE
:1038B000080EDBCF15F0153404E21450FF08000E9B
:1038C000155404E2070EDB68080EDB6A0101425161
:1038D000EA6A980FE96E000EEA22070EDBCFEFFFCF
:1038E00036D04251EA6A980FE96E000EEA22EFCF15
:1038F00009F0DFCF0EF0B0EC1EF009C0EFFF27D0CB
:10390000DF1CE66E4251EA6A980FE96E000EEA2269
:10391000E552E750EF6E1BD04251EA6A980FE96E0C
:10392000000EEA22DF50EF1612D04251EA6A980FD9
:10393000E96E000EEA22DF50EF1209D04251EA6A26
:10394000980FE96E000EEA22DF50EF1A00D044C152
:103950009AF0090EE15C02E2E16AE552E16EE5529D
:06396000E7CFD9FF1200C1
:0A396600020120511F0B010801E0CF
:103970006DD0245101E06AD0060E215D28E123516B
:10398000230A21E0010A11E0030A01E020D000012E
:10399000C0050AE10001760ED06F3A0ED16F090E14
:1039A000D36FD46BC00ED26F12D00001C0050AE1F4
:1039B0000001F30ED06F3A0ED16F1D0ED36FD46B92
:1039C000C00ED26F04D00001800ED26F00D0020171
:1039D0002051600BE842E842E842E842E842010830
:1039E00001E034D021510B0A2BE0080A1EE0090A3D
:1039F00016E0080A09E00B0A05E0080A01E026D0F3
:103A000026D824D025D822D00001490ED06F010E2F
:103A1000D16F010ED36FD46BC10ED26F17D00001DE
:103A2000800ED26F23C249F111D000014A0ED06F2F
:103A3000010ED16F010ED36FD46B810ED26F06D001
:103A40000001800ED26F22C24AF100D01200120093
:023A5000120062
:0E3A52001201000200000008621900200101AC
:103A60000102000109022900010100C0320904001D
:103A7000000203000000092111010001221D0007BE
:103A8000058103400001070501034000010403090B
:103A90000434035600730074006F006E006500204C
:103AA0000043006F002E002C004C00740064002EB8
:103AB0000020002000200020002000200020002006
:103AC00000200020002E0342006500610075007494
:103AD000006F00200053007400690063006B002039
:103AE0000048004900440020002000200020002061
:103AF0000020000600FF0901A1011901294015005D
:103B000026FF00750895408102190129409102C0E5
:083B1000643A8D3A913AC53A7E
:083B18001E0EF66E100EF76E92
:103B2000000EF86E00010900F550FB6F0900F5501A
:103B3000FC6F03E1FB6701D03DD00900F550F66F43
:103B40000900F550F76F0900F550F86F09000900FA
:103B5000F550E96E0900F550EA6E09000900090008
:103B6000F550F96F0900F550FA6F09000900F6CF1A
:103B7000FDF0F7CFFEF0F8CFFFF0F6C0F6FFF7C08C
:103B8000F7FFF8C0F8FF0001F95302E1FA5307E02C
:103B90000900F550EE6EF907F8E2FA07F9D7FDC013
:103BA000F6FFFEC0F7FFFFC0F8FF0001FB07000EA5
:063BB000FC5BBFD7120010
:0A3BB60006500B02F3CF02F0F4CF2B
:103BC00003F00C02F3500326000EF420046E06509E
:103BD0000D02F3500426000EF420056E06500E026E
:103BE000F350052607500B02F3500326F45004222D
:103BF000000E052207500C02F3500426F450052253
:103C000007500D02F350052608500B02F35004260E
:103C1000F450052208500C02F350052609500B02FF
:063C2000F350052612001E
:0A3C260009C013F008C012F00850A6
:103C30000D02F4CF07F0F3CF06F009500E02F4CFD7
:103C400009F0F3CF08F00D02F3500726F4500822D4
:103C5000E86A092212500E02F3500726F450082297
:103C6000E86A09220EAE39EF1EF01250085E1350BA
:103C7000095A13AE000C0D50085E0E50095A000C84
:103C8000D9CFE6FFE1CFD9FFE6527F6A938A939EB0
:103C9000240EAC6E900EAB6E710EAF6E020EB06E57
:103CA000080EB86EAE50DF6EE552E552E7CFD9FF91
:103CB0001200D9CFE6FFE1CFD9FFFE0EDB50AD6E8B
:083CC000E552E7CFD9FF120025
:083CC800056A046A036A026A3E
:103CD000200EE76ED89006360736083609360236CB
:103CE0000336043605360B50025C0C5003580D5059
:103CF00004580E50055809E30B50025E0C50035A4D
:103D00000D50045A0E50055A062AE72EE4D7120029
:103D1000FE0EE3CFE9FFFF0EE3CFEAFFE9CFF3FFAB
:103D2000EACFF4FFFB0EE35003E1FC0EE35009E0A1
:103D3000FB0EE30602E2FC0EE306FD0EE350EE6E20
:043D4000F1D71200A5
:0C3D440011EE00F021EE00F0F86A019C86
:103D50008CEC1DF003EC08F0ABEC08F0FBD7120084
:103D6000056A080EE76ED890093605360E50055CD8
:0C3D700002E3056E092AE72EF7D71200C7
:043D7C0000EE00F065
:0A3D80000F0EEE6AEA62FDD7120092
:063D8A0015CD5B07E555B5
:0C3D90009A15B53B121F331349050000C3
:043D9C001100000012
:103DA0000000FFFF0000FFFFFFFFFF000000FFFF1C
:103DB000FFFFFFFFFFFFFFFFFFFFFFFF000000000F
:103DC00001000000000000000000000000000000F2
:043DD00000000000EF
:00000001FF
